:100000002F2883178001840AFF3E031D02282A2817
:10001000A301A200FF30A207031CA307031C2A2888
:100020000330A100DF3016200A28A101E83EA0001D
:10003000A109FC30031C1F28A00703181C28A007D7
:100040000000A10F1C2820182528A01C292800002A
:1000500029280800831383120313000008000730C7
:100060009F000C30831685005030860020308400BD
:10007000603083120220A0308400503002202030F3
:1000800084003030012005120610861006118611FA
:1000900005108510051385138613A5018612722895
:1000A000A7010530A6000230A300BC3009200512CC
:1000B0000610861006118611061A6828A603260A5D
:1000C0000319A70327082604031D6828A501722821
:1000D0000230A300BC30092005160614861406154C
:1000E0008615532886170130A300F4300920051720
:1000F0000330A300E830092085170530A300DC3069
:10010000092005140730A300D030092085140530DC
:10011000A400061AA828A408031D90287228A8285D
:100120004B30A700A60186160430A000A00B96282D
:10013000000086120430A000A00B9C2800000130B3
:10014000A6020318A428A70203189328A403861262
:1001500005302402031DAF2801300820CB280430CD
:100160002402031DB5288510CB2803302402031D6B
:10017000BB280510CB2802302402031DC12885139B
:10018000CB2801302402031DC7280513CB28A4085F
:10019000031DCB288613061BD728A408031DD228CD
:1001A0007228D728A50A0130A300F43009200130B5
:1001B0002502031DDD280516F92802302502031D3E
:1001C000E3280614F92803302502031DE9288614C4
:1001D000F92804302502031DEF280615F9280530FB
:1001E0002502031DF92886150130A300F4300920EB
:0801F000502889286300FA2859
:02400E00503F21
:00000001FF
